:100000000C9434000C9451000C9451000C94510049
:100010000C9451000C9451000C9451000C94E50088
:100020000C9451000C9451000C9451000C94B400A9
:100030000C9451000C9451000C9483000C945100CA
:100040000C9451000C9451000C9451000C945100EC
:100050000C9451000C9451000C9451000C945100DC
:100060000C9451000C94510011241FBECFEFD8E026
:10007000DEBFCDBF11E0A0E0B1E0ECE1F6E002C0F0
:1000800005900D92A231B107D9F711E0A2E1B1E0DC
:1000900001C01D92A731B107E1F70E9445010C9400
:1000A0000C030C9400008230910561F083309105BF
:1000B00099F00197C9F416BC80916E00826080931C
:1000C0006E0016C0109285001092840080916F001F
:1000D000826080936F000CC01092B200809170001B
:1000E00082608093700004C081E090E00E940C0365
:1000F00078949FB7F894809114019FBF8823C9F327
:100100001092140108951F920F920FB60F921124AE
:100110002F933F938F939F9380911201909113019E
:100120000196909313018093120180911401813004
:1001300091F020911201309113018091150190915D
:1001400016012817390738F081E0809314011092C6
:100150001301109212019F918F913F912F910F9057
:100160000FBE0F901F9018951F920F920FB60F920F
:1001700011242F933F938F939F938091120190911D
:100180001301019690931301809312018091140141
:10019000813091F02091120130911301809115016D
:1001A000909116012817390738F081E080931401E7
:1001B00010921301109212019F918F913F912F91F4
:1001C0000F900FBE0F901F9018951F920F920FB6B1
:1001D0000F9211242F933F938F939F93809112013D
:1001E00090911301019690931301809312018091D5
:1001F0001401813091F0209112013091130180910E
:100200001501909116012817390738F081E0809385
:10021000140110921301109212019F918F913F913E
:100220002F910F900FBE0F901F901895FC01A1E821
:10023000B0E08C918D608C9382E090E09387828710
:10024000229AA0E8B0E08C9181628C93AAE8B0E099
:1002500011961C921E921C92B587A48785B5836067
:1002600085BD81E090E0978786872AE030E0309373
:1002700016012093150124B5226024BD29EF27BD66
:10028000918B808B80E090E00895CF92DF92EF9287
:10029000FF9280E091E00E941601C12CD12C7601E2
:1002A00060E070E0CB0160930001709301018093E6
:1002B00002019093030120E030E040E85FE30E94F8
:1002C000F30187FF03C08FEF90E002C080E090E071
:1002D0009093050180930401809110019091110188
:1002E0000E945300E0910C01F0910D0180910401F6
:1002F00080838FEFC81AD80AE80AF80AC701B60146
:100300000E94F7012FE632E143E05BE30E94A9027D
:1003100020E030E0A9010E948F01C5CF5058BB27D3
:10032000AA270ED0DCC0CDD030F0D2D020F031F4EE
:100330009F3F11F41EF4C2C00EF4E095E7FBB8C075
:10034000E92FDED080F3BA17620773078407950799
:1003500018F071F49EF5F6C00EF4E0950B2EBA2F4E
:10036000A02D0B01B90190010C01CA01A0011124BB
:10037000FF27591B99F0593F50F4503E68F11A1667
:10038000F040A22F232F342F4427585FF3CF4695F8
:1003900037952795A795F0405395C9F77EF41F161A
:1003A000BA0B620B730B840BBAF09150A1F0FF0FE4
:1003B000BB1F661F771F881FC2F70EC0BA0F621FD0
:1003C000731F841F48F4879577956795B795F795C0
:1003D0009E3F08F0B3CF9395880F08F09927EE0F52
:1003E00097958795089540D008F481E00895E894A2
:1003F00009C097FB3EF490958095709561957F4F6D
:100400008F4F9F4F9923A9F0F92F96E9BB2793951A
:10041000F695879577956795B795F111F8CFFAF42A
:10042000BB0F11F460FF1BC06F5F7F4F8F4F9F4F5B
:1004300016C0882311F096E911C0772321F09EE8B9
:10044000872F762F05C0662371F096E8862F70E01F
:1004500060E02AF09A95660F771F881FDAF7880FF9
:100460009695879597F90895990F0008550FAA0B4F
:10047000E0E8FEEF16161706E807F907C0F01216B7
:100480001306E407F50798F0621B730B840B950BBA
:1004900039F40A2661F0232B242B252B21F408950F
:1004A0000A2609F4A140A6958FEF811D811D0895AC
:1004B00097F99F6780E870E060E008959FEF80EC17
:1004C000089500240A9416161706180609060895BA
:1004D00000240A9412161306140605060895092E20
:1004E0000394000C11F4882352F0BB0F40F4BF2B8F
:1004F00011F460FF04C06F5F7F4F8F4F9F4F0895CF
:1005000057FD9058440F551F59F05F3F71F04795C4
:10051000880F97FB991F61F09F3F79F087950895A9
:10052000121613061406551FF2CF4695F1DF08C0C8
:10053000161617061806991FF1CF869571056105E5
:1005400008940895E894BB2766277727CB0197F98D
:1005500008950BD0C4CFB5DF28F0BADF18F095238B
:1005600009F0A6CFABCF1124EECFCADFA0F3959F41
:10057000D1F3950F50E0551F629FF001729FBB278A
:10058000F00DB11D639FAA27F00DB11DAA1F649F36
:100590006627B00DA11D661F829F2227B00DA11DE9
:1005A000621F739FB00DA11D621F839FA00D611D6F
:1005B000221F749F3327A00D611D231F849F600D90
:1005C000211D822F762F6A2F11249F5750408AF0C9
:1005D000E1F088234AF0EE0FFF1FBB1F661F771F55
:1005E000881F91505040A9F79E3F510570F060CF91
:1005F000AACF5F3FECF3983EDCF38695779567953D
:10060000B795F795E7959F5FC1F7FE2B880F911D72
:0C0610009695879597F90895F894FFCF10
:10061C0000000000FF000AD7233C0000000000008F
:02062C000000CC
:00000001FF
